:100000000C9476060C9493060C9493060C94930629
:100010000C9493060C9493060C9493060C949306FC
:100020000C9493060C9493060C94B82C0C948A2D83
:100030000C9479260C9493060C9493060C949306D6
:100040000C9493060C9493060C9493060C949306CC
:100050000C9493060C9402270C9493060C9493062C
:100060000C9493060C9493060C9493060C949306AC
:100070000C9493060C9493060C9493060C9493069C
:100080000C9493060C9493060C9493060C9493068C
:100090000C9493060C9493060C9493060C9493067C
:1000A0000C9493060C9493060C9493069F0A9F0A53
:1000B000CB0ACB0A2C0B4A0B280C280C4F0BB70B86
:1000C000C80BC80B781DEA1D801D4A1D4E1D841DDE
:1000D000511D871D921D5C1DE01D601D961D641D38
:1000E0009A1DC41D681D9E1DCE1D6E1DA41DAE1D36
:1000F000551D8B1D581D8E1D731DA91DBA1DDA1DA2
:10010000DC1D461D7C1DF31DC922CF22BD22C3224A
:10011000D522DB22E122DE23E12318242B24332401
:100120003E2441244124412489248924462449240D
:100130004E245B2468246B246F247C24F22D192E1A
:10014000112F192E112F652E882E112FDF2EEE2E36
:10015000415254005500560001000000000000000C
:1001600000000000000000000000000000005F0030
:100170006000610057000100000000000000000066
:100180000000000000000000000000005C005D00B6
:100190005E005700010000000000000000000000A9
:1001A0000000000000000000000059005A005B0041
:1001B00058000100000000000000000000000000E6
:1001C00000000000000000006200620063005800B0
:1001D000010000000000000000000000000000001E
:1001E00000000000000001001E001F002000210090
:1001F0002200230024002500260027000100010022
:1002000001000100290014001A0008001500170061
:100210001C0018000C00120013002A005F00600090
:1002200061002B0004001600070009000A000B0003
:100230000D000E000F00330034005C005D005E0016
:10024000E1001D001B000600190005001100100050
:10025000360037003800282259005A005B00E000C1
:10026000E300E200E2002252E1002C002352E7000A
:10027000E6004C00E400620062006300010001003F
:100280000100010001000100010001000100010066
:100290000100010001000100010001003A003B00E3
:1002A0003C003D003E003F00400041004200430052
:1002B000530054005500560035001E001F0020005A
:1002C0002100220023002400250026002700010031
:1002D0000100010057000100440045000100010039
:1002E00001002800E500E70037242A210100010071
:1002F000010058000100010001000100010001009F
:100300002800E500010001000100010001000100DA
:1003100001000100010001000100010001000100D5
:1003200001000100010001000100010001000100C5
:10033000007C2B00520001004900E000E1004B006E
:100340004A002D002E004C00010001000100390080
:10035000500051004F004600E100E0004E004D000B
:100360002F003000310001000100010001004800B1
:10037000010001000100010001000100E700E600AA
:1003800001000100010001000100405201000100D4
:100390000100010001000100010001000100010055
:1003A000010001000100010044454255473A206424
:1003B000697361626C65642E0A0044454255473A90
:1003C00020656E61626C65642E0A006C65645F7402
:1003D00061736B3A20253032580A004F6E6573689E
:1003E0006F743A206163746976653A2025640A0067
:1003F0000A002530313662003A200025303258009C
:100400000A722F6320303132333435363738394170
:1004100042434445460A00313A0964656C617928D3
:100420002A31306D73293A2025750A323A09696EEE
:1004300074657276616C286D73293A2025750A33CC
:100440003A096D61785F73706565643A2025750AB5
:10045000343A0974696D655F746F5F6D61783A2035
:1004600025750A353A09776865656C5F6D61785F57
:1004700073706565643A2025750A363A09776865B0
:10048000656C5F74696D655F746F5F6D61783A204C
:1004900025750A00703A097072696E742076616C75
:1004A0007565730A643A09736574206465666175DD
:1004B0006C74730A75703A092B310A646E3A092D0F
:1004C000310A6C743A092B31300A72743A092D31B1
:1004D000300A4553432F713A09717569740A0A73DA
:1004E00070656564203D2064656C7461202A206D10
:1004F00061785F7370656564202A20287265706575
:100500006174202F2074696D655F746F5F6D617811
:10051000290A77686572652064656C74613A2063A6
:100520007572736F723D25642C20776865656C3D2C
:1005300025640A53656520687474703A2F2F656EC0
:100540002E77696B6970656469612E6F72672F77AA
:10055000696B692F4D6F7573655F6B6579730A0001
:100560004D3E20004D25753A25733E20003F0A0080
:100570003D2025750A003F0A0064656661756C744C
:10058000730A0025750A003F0A000A092D205661EA
:100590006C756573202D0A00710A000A092D204D23
:1005A0006F7573656B6579202D0A003F00433E200F
:1005B000004C25640A000A092D2053746174757378
:1005C000202D0A686F73745F6B6579626F61726466
:1005D0005F6C65647328293A20253032580A6B65B0
:1005E00079626F6172645F70726F746F636F6C3A7F
:1005F00020253032580A6B6579626F6172645F69D9
:10060000646C653A20253032580A74696D65725FF2
:1006100072656164333228293A202530386C580AD3
:10062000002573000A092D20436F6E736F6C6520DF
:100630002D0A4553432F713A09717569740A6D3A51
:10064000096D6F7573656B65790A000A092D204D78
:1006500061676963202D0A443A0944656275672021
:100660004D65737361676520546F67676C650A58E1
:100670003A094D6174726978204465627567204D4E
:100680006F646520546F67676C65202D2053686F19
:1006900077206B65797072657373657320696E205E
:1006A0006D617472697820677269640A4B3A094B0C
:1006B0006579626F61726420446562756720546F6A
:1006C00067676C65202D2053686F77206B657970A4
:1006D00072657373207265706F72740A4D3A0944C3
:1006E00065627567204D6F75736520546F67676C21
:1006F000650A563A0956657273696F6E0A533A096C
:100700005374617475730A433A094163746976617D
:10071000746520436F6E736F6C65204D6F64650A5E
:1007200046312D4631303A09537769746368207435
:100730006F204C6179657220302D39202846313088
:10074000203D204C30290A302D393A0953776974FD
:10075000636820746F204C6179657220302D390AEE
:1007600047524156453A0953776974636820746F5C
:10077000204C6179657220302028616C7465726E3E
:10078000617465290A423A094A756D7020746F20B8
:10079000426F6F746C6F616465720A4553433A0926
:1007A0004A756D7020746F20426F6F746C6F616456
:1007B00065722028616C7465726E617465290A45E2
:1007C0003A095072696E7420454550524F4D20537E
:1007D000657474696E67730A4241434B53504143D9
:1007E000453A09436C65617220454550524F4D0AA8
:1007F000006B65796D61705F636F6E6669672E72FD
:1008000061773A20253032580A2E737761705F6322
:100810006F6E74726F6C5F636170736C6F636B3A51
:100820002025750A2E636170736C6F636B5F746F44
:100830005F636F6E74726F6C3A2025750A2E737742
:1008400061705F6C63746C5F6C6775693A202575C5
:100850000A2E737761705F7263746C5F726775697B
:100860003A2025750A2E737761705F6C616C745F36
:100870006C6775693A2025750A2E737761705F720F
:10088000616C745F726775693A2025750A2E6E6F08
:100890005F6775693A2025750A2E737761705F6707
:1008A000726176655F6573633A2025750A2E7377EA
:1008B00061705F6261636B736C6173685F626163D7
:1008C0006B73706163653A2025750A2E6E6B726FCB
:1008D0003A2025750A2E737761705F6573636170C6
:1008E000655F636170736C6F636B3A2025750A00F6
:1008F00064656275675F636F6E6669672E726177A4
:100900003A20253032580A2E656E61626C653A20B5
:1009100025750A2E6D61747269783A2025750A2E44
:100920006B6579626F6172643A2025750A2E6D6F6E
:100930007573653A2025750A006565636F6E666993
:10094000673A0A64656661756C745F6C617965729B
:100950003A2025750A003F000A6D6F7573653A20CD
:100960006F66660A000A6D6F7573653A206F6E0ACE
:10097000000A6B6579626F6172643A206F66660A7D
:10098000000A6B6579626F6172643A206F6E0A00CB
:100990000A6D61747269783A206F66660A000A6DA2
:1009A00061747269783A206F6E0A000A6465627534
:1009B000673A206F66660A000A64656275673A20C6
:1009C0006F6E0A000A0A4A756D70696E6720746F4F
:1009D00020626F6F746C6F616465722E2E2E200022
:1009E000433E2000436C656172696E672045455047
:1009F000524F4D0A00290A002575002F0025750069
:100A00005D28002564002000256400200025640086
:100A100020002564007C0025303258006D6F75730E
:100A2000656B6579205B62746E7C78207920762016
:100A3000685D287265702F61636C293A205B000045
:100A4000000000000000002A2B2800000000000029
:100A50000000000000000000000029000000002C41
:100A60001E3420212224342627252E362D373827E0
:100A70001E1F202122232425263333362E37381FEC
:100A80000405060708090A0B0C0D0E0F10111213AE
:100A90001415161718191A1B1C1D2F3130232D354C
:100AA0000405060708090A0B0C0D0E0F101112138E
:100AB0001415161718191A1B1C1D2F3130354C0030
:100AC0000000000000000000000000000000000026
:100AD0000000000000000000000000000000000016
:100AE0000000007E0F00D4FFFFFFC7000000780A5F
:100AF000002530325820006B6579626F6172645F47
:100B00007265706F72743A2025303258207C200054
:100B100073757370656E64696E67206B6579626F5B
:100B20006172640D0A005B575D005B535D005B52B0
:100B30005D005B445D005B435D0022035400680080
:100B40006500200035007800350020004B0065006E
:100B5000790062006F0061007200640000000C0305
:100B600064006900300069006200000004030904A9
:100B700009027400040100A0FA0904000001030145
:100B80000100092111010001224400070581030829
:100B90000001090401000203000000092111010005
:100BA000012222000705820320000107050303201C
:100BB00000010904020001030000000921110100E5
:100BC00001227B00070584032000010904030001C2
:100BD000030000000921110100012215000705850D
:100BE0000320000112010002000000082540B505A5
:100BF0000001010200010631FF0974A10109751508
:100C00000026FF00952075088102C00660FF09617B
:100C1000A1010962150026FF0095207508810209CF
:100C200063150026FF00952075089102C005010993
:100C300002A10185020901A1000509190129081570
:100C4000002501950875018102050109300931155A
:100C500081257F95027508810609381581257F95C4
:100C60000175088106050C0A38021581257F95015A
:100C700075088106C0C005010980A101850319011D
:100C80002AB700150126B700950175108100C0052F
:100C90000C0901A101850419012AA002150126A051
:100CA00002950175108100C005010906A101050723
:100CB00019E029E7150025019508750181029501C4
:100CC000750881010507190029FF150026FF009509
:100CD00006750881000508190129051500250195EB
:100CE0000575019102950175039101C011241FBE84
:100CF000CFEFDAE0DEBFCDBF12E0A0E0B1E0E0E48C
:100D0000F0E602C005900D92A23EB107D9F723E0AC
:100D1000A2EEB2E001C01D92A83CB207E1F70E942A
:100D2000AC170C941E300C940000FF93EF93E091ED
:100D3000E202F091E302309709F00995EF91FF91FB
:100D40000895FC018591803011F0EFDFFBCF08950D
:100D5000FF27E0E230E247FF0CC0419597FF09C052
:100D6000EDE26095709580959095611D711D811DD6
:100D7000911D27FF02C0219530E350E2AA27660F9C
:100D8000771F881F991FAA1FA41710F0A41B639533
:100D90005A95A9F7AA3008F0A95FA05DAF93F39523
:100DA000611571058105910541F7ED3211F4EF935D
:100DB000F395F21718F43F93F395FBCF8F91B5DFBE
:100DC000FA95E1F70895E991F9918591803021F044
:100DD000853219F0AADFF9CF089520E0E894559103
:100DE0005532C1F3503311F4689455915A3348F495
:100DF000505390F3220F022E220F220F200D250FA9
:100E0000F4CF0EF4219589919991533619F3533704
:100E100029F1533559F1BC0188279927E8945C36AC
:100E200021F48991999168945591543639F446EF9B
:100E30007EF077FF0DC08FEF9FEF0AC055374AE075
:100E400039F0583540E121F0523642E009F008957A
:100E5000FF93EF937DDFEF91FF91B7CFFF93EF9378
:100E6000FC0181918030B9F360DFFBCFFF93EF93FA
:100E700068DFF1CFDF93CF93CDB7DEB72596A3DF41
:100E8000CF91DF9108958430B0F46530A0F44F30F5
:100E900090F49BE4899FF00111248FE0689FE00D9E
:100EA000F11D1124E40FF11DEE0FFF1FE05BFE4F5B
:100EB00085919491089581E090E0089581E00895EE
:100EC00081E008950E94600708950E9462070895D6
:100ED0000E946007089508950E946B070895A6E098
:100EE000B0E0E5E7F7E00C947A2F49835A839E83BC
:100EF0003091E90289819A81311115C03E813323F5
:100F000059F0222349F00E94C20D182F682F8981C1
:100F10009A810E949E0D03C00E94B00D182F698116
:100F20007A81812F04C00E94C20D69817A810E945A
:100F300001152696E3E00C94962FFC01262F4081A4
:100F4000518162817381848195810E946F07089528
:100F5000CF93DF93EC0161E00E949D07BE010E94E8
:100F60006507DF91CF910895CF93DF93EC0160E0A7
:100F70000E949D07BE010E946C07DF91CF910895EA
:100F800091E001C0990F8A95EAF7892F0E94E70C3A
:100F90000895CF93C82F81E00C2E01C0880F0A94CA
:100FA000EAF70E9452128C2F0E94C007CF91089539
:100FB00081E008950E94D8070895CF93C82F0E941A
:100FC000990C8C2F0E94DA072FEF84E39CE02150CC
:100FD00080409040E1F700C00000CF91089581E08B
:100FE0000E94DD070E942827089580E00E94DD0707
:100FF0000E94392708950F931F93CF93DF938C019D
:1010000061E00E949D07EC01B8010E94AB23882398
:10101000C1F1B801CE010E946807882391F1B8019F
:10102000CE010E94B122882361F1B801CE010E9455
:10103000221D882331F1B801CE010E94F81C8823BB
:1010400001F1B801CE010E94F4228823D1F0B80149
:10105000CE010E94FD158823A1F0F8018581882327
:1010600009F446C0C3308CE7D807C1F160F4C13041
:10107000FCE7DF07A9F1A8F4C115DC47C9F50E9418
:10108000EF07C0E039C0CB35FCE7DF0779F1CC359D
:101090008CE7D80741F1CA35DC4751F50E942D1283
:1010A00027C080917403C82FC095C170C0FB80F920
:1010B00080937403CC2349F08AEB93E09F938F9342
:1010C0000E943A070F900F90DCCF88EA93E09F933D
:1010D0008F930E943A070F900F900EC00E94351216
:1010E0000E94F507CECF0E94231202C00E94311247
:1010F000C8010E945E07C82F8C2FDF91CF911F91EE
:101100000F9108950E9451260E94C70808950E94D9
:10111000CB080E945A2608958295982F937344E035
:10112000949F900111248C7C86958695282B822F84
:101130008575880F2A7A2695822B0895CF93DF93A1
:10114000D92F0E948C08C82F8D2F0E948C082C2F1D
:1011500030E0322F2227A901482BCA01DF91CF911D
:10116000089581E008950895CF93DF93D82F0E94CA
:10117000B108C82F882319F08D2F0E94B3088C2F37
:10118000DF91CF91089508950E94B408089580E0FA
:101190000E94C40808950E9499240E94C4080895DA
:1011A000CF930E949924C82F8091E402C81709F1B7
:1011B000C093E4020E94E7266093E5027093E60282
:1011C0008093E7029093E8028091740382FF0EC03F
:1011D00080FF0CC01F92CF938BEC93E09F938F9373
:1011E0000E943A070F900F900F900F908C2F0E9443
:1011F000C408CF910895ADE0B0E0E1E0F9E00C94CF
:101200007B2F488759876A877B878C879D879111B9
:101210000E944B11CE01019627E0FC0111922A9504
:10122000E9F726E0FE013896DC0101900D922A953F
:10123000E1F72D8121110AC029813A814B815C811E
:101240006D817E818F810E94951004C00E94A80745
:101250008111F2CF2D96E2E00C94972FFC012481AE
:10126000213021F4808191810E94EF0D0895662341
:1012700019F00E94921E02C00E94ED1E0E94641F7F
:101280000895CF93882309F48DC0C82F8238A1F424
:101290000E94A62481FD86C089E30E9498250E94B1
:1012A000AD112FEF87EE93E0215080409040E1F7A1
:1012B00000C0000089E315C08338C1F40E94A62451
:1012C00080FD70C083E50E9498250E94AD112FEF2C
:1012D00081EE94E0215080409040E1F700C0000092
:1012E00083E50E94A0250E94AD115CC08438A1F462
:1012F0000E94A62482FD56C087E40E9498250E9481
:10130000AD112FEF81EE94E0215080409040E1F745
:1013100000C0000087E4E5CF8CEF8C0F813A98F491
:101320008C2F0E94FD1A81113DC08C2F0E945D25DB
:10133000882329F08C2F0E94A0250E94AD118C2FAC
:101340000E949825D0CF80E28C0F883048F4C77077
:1013500081E001C0880FCA95EAF70E942E11C3CF21
:10136000EBE5EC0FE33040F4F0E0EF5AFE4F808104
:1013700090E00E94042516C0E8E5EC0FEB3150F434
:10138000F0E0EE0FFF1FE55EFE4F808191810E942D
:10139000292508C083E38C0F833120F461E08C2F72
:1013A0000E943709CF910895882309F456C08238E6
:1013B00059F40E94A62481FF50C089E30E94982519
:1013C0000E94AD1189E30CC0833879F40E94A624F1
:1013D00080FF43C083E50E9498250E94AD1183E5FC
:1013E0000E94A0250E94AD110895843859F40E94EE
:1013F000A62482FF32C087E40E9498250E94AD1186
:1014000087E4EECF9CEF980F913A50F390E2980F5B
:10141000983050F4877091E001C0990F8A95EAF7EF
:10142000892F0E943411DECF9BE5980F933028F46A
:1014300080E090E00E940425089598E5980F9B3184
:1014400028F480E090E00E942925089593E3980F06
:10145000933118F460E00E94370908951F93CF93E9
:10146000DF93182FEB010E944109209741F08FE98B
:101470009FE00197F1F700C000002197F6CF812F80
:101480000E94D409DF91CF911F910895893319F0FB
:1014900060E070E002C060E570E00E942E0A0895EE
:1014A000882321F00E942E110E94AD1108958823F7
:1014B00021F00E9434110E94AD110895A0E0B0E027
:1014C000E4E6FAE00C94752F7C01162FC72FFC017F
:1014D000D581068102950F700E9424118823F9F0AE
:1014E000DD23E9F08C2F807F803461F080E2810F72
:1014F0008830A8F08C2F807E803221F4123078F072
:10150000002369F08091A20382FF09C082E00E945B
:10151000E3110E94241191E0D82ED92601C0D12CCC
:10152000CC2EC2948FE0C8228C2D90E08C30910597
:1015300008F08EC1FC01EA5AFF4F0C945E2F8C2FED
:10154000807FCF70882311F0C295C07FDD2399F092
:10155000CC2309F469C180E2810F883010F01111A9
:1015600004C08C2F0E942E1103C08C2F0E943E11AC
:101570000E94AD1159C1812F0E94D409CC2309F4D6
:1015800067C180E2810F883038F1112329F18C2F57
:101590000E94441124C08C2F807FCF70803211F0C4
:1015A000C295C07F112319F0113099F13CC0809190
:1015B000A20382FD17C0DD2349F0CC2329F08C2F34
:1015C0000E942E110E94AD1180E02FC180E00E9488
:1015D000D409CC2309F43CC18C2F0E9434110E9401
:1015E000AD1136C1DD2349F0002309F1013009F0C6
:1015F0002FC18C2F0E9455112BC1011129C18C2F95
:101600000E94570A8C2F0E9461118C2F0E94B611E4
:101610001FC1DD2321F0063008F01AC108C00530D3
:1016200008F016C115C0DD2331F00111FDC08C2F6B
:101630000E94500A0DC1002359F0193309F005C169
:10164000FFEF27EE83E0F15020408040E1F7FBC040
:101650008C2F0E94570AFCC08C2F8695869583702C
:1016600019F0813061F0F4C0DD2321F0812F9C2F2F
:10167000937002C080E090E00E940425F1C0DD2359
:1016800021F0812F9C2F937002C080E090E00E9497
:101690002925E6C06D2F812F0E943709E1C08C2FCC
:1016A000837079F5D111D8C0412F42954695477086
:1016B000440F440F212F2F70042E01C0220F0A94D3
:1016C000EAF714FF08C08FE090E001C0880F4A9548
:1016D000EAF7809501C080E0C695C695C370822B5D
:1016E000C23049F058F4C13019F00E94F00CB4C077
:1016F0000E94EA0CB1C00E94F60CAEC00E94E70C3A
:10170000ABC0DD2319F08C2F817001C08695882332
:1017100009F4A2C0412F429546954770440F440FEB
:10172000212F2F70042E01C0220F0A94EAF714FF14
:1017300008C08FE090E001C0880F4A95EAF78095D5
:1017400001C080E0C695C695C370822BC23049F0B7
:1017500058F4C13019F00E943C0D7EC00E94360D35
:101760007BC00E94420D78C00E94FF0C75C0CF70F4
:10177000DD2339F08C2F0E94110D812F0E94500A19
:101780006BC0812F0E94570A8C2F0E941D0D64C0D0
:10179000123F21F128F4103F41F0113FC1F040C049
:1017A000133F19F1143F79F03BC0DD2341F00530C0
:1017B00008F04EC08C2F8F710E942A0D49C0063050
:1017C00008F046C0F7CF8091A20382FD18C0DD2348
:1017D00039F08C2F8F710E94110D3AC0DD23C9F3AF
:1017E0008C2F8F710E941D0D33C0DD2329F08C2FAB
:1017F0008F710E94080D2CC00E94040D29C0DD23AA
:1018000031F063E08C2F8F710E94C51121C081E0FF
:101810000E94E3110230E0F082E00E94E31118C060
:10182000DD2331F00023A9F2812F0E94410910C06D
:101830000023B1F2193349F49FEFE7EEF3E0915042
:10184000E040F040E1F700C00000812F0E94D40981
:1018500088EF8C0D843020F40E9499240E94C408E3
:10186000DD2089F00E94201180FD0DC0F701158256
:101870000E941A110E94110DC7010E94600C0E9463
:101880001A110E941D0DCDB7DEB7E8E00C94912F20
:101890000F931F93CF93DF93EC01688179818D8142
:1018A0000E94FA0D8C010E94480D0E94DA0CB801CA
:1018B000CE010E945E0ADF91CF911F910F91089592
:1018C000CF93DF93FC0124812223D1F0EC010E940D
:1018D000FB0781110FC00E942411882389F08D819C
:1018E000882371F08091A20382FF0AC082E00E94E7
:1018F000E31106C0CE010E94480CCE010E94B4073D
:10190000DF91CF91089580E090E00E94042580E06F
:1019100090E00E9429250E944B110E94AD110E9467
:101920001D200E94641F08950E94A8250E94830C18
:1019300008950E943B110E94940C089592959F7007
:10194000963079F010F4925001C09A50923068F4B9
:10195000803F69F018F4883E40F409C0843F29F4C0
:1019600006C0883E20F0813F11F080E0089581E0BC
:101970000895FC012481222339F0808191810E9405
:10198000EF0D0E949E0C089580E00895A6E0B0E05F
:10199000ECECFCE00C947B2F2696E2E00C94972F65
:1019A000A7E0B0E0E6EDFCE00C947B2F2796E2E0A8
:1019B0000C94972F089508950E94DB0C08950E94BF
:1019C000DC0C08950E94DF0C8093090308950E94A7
:1019D000E20C089590910903892B0E94E20C08956E
:1019E0009091090389230E94E20C089590910903C4
:1019F00089270E94E20C08950E94DB0C08950E9442
:101A0000FC0C80930803089580E00E94FF0C089569
:101A100091E001C0990F8A95EAF7892F0E94FF0C87
:101A2000089521E030E001C0220F8A95EAF7809105
:101A30000803822B0E94FF0C089521E030E001C0D2
:101A4000220F8A95EAF720958091080382230E944D
:101A5000FF0C089521E030E001C0220F8A95EAF7DB
:101A60008091080382270E94FF0C0895909108033B
:101A7000892B0E94FF0C08959091080389230E94EE
:101A8000FF0C08959091080389270E94FF0C089588
:101A90000895962F9770A1E001C0AA0F9A95EAF7D2
:101AA00093E0769567959A95E1F7FB01EE0FFF1F9E
:101AB0006E0F7F1FFA01E60FF71F40E050E0682F1E
:101AC00070E090819B01042E02C0369527950A9400
:101AD000E2F72170219529272A23292721934F5F97
:101AE0005F4F4330510569F708959B01782F777058
:101AF00043E0969587954A95E1F7FC01EE0FFF1FAD
:101B00008E0F9F1FF901E80FF91F40E050E080E0C1
:101B1000219130E0072E02C0369527950A94E2F70E
:101B200021703327042E01C0220F0A94EAF7822B7A
:101B30004F5F5F4F4330510559F70895282F953077
:101B400070F48F3060F4862F622F70E02FE0929F48
:101B5000600D711D11244AEE52E00E94490D089556
:101B6000953070F48F3060F4292F90E06AEE72E0C7
:101B70003FE0239F800D911D11240E94750D089553
:101B800080E00895CF92DF92FF920F931F93CF933F
:101B9000DF936C010091080380910903082BC3E0D7
:101BA000D0E010E0C8010C2E02C0959587950A94EC
:101BB000E2F780FD04C02197A8F7F12C07C0FC2EA6
:101BC000B6018C2F0E940D150197A9F38F2DDF917F
:101BD000CF911F910F91FF90DF90CF900895CF93F9
:101BE000DF93EC010E94C20DBE010E940D15DF9132
:101BF000CF9108951F93CF93DF93EB019091E9026A
:101C0000992321F0CB010E94EF0D13C0882349F0E6
:101C1000CB010E94C20D182F682FCE010E949E0D8D
:101C200004C0CB010E94B00D182FBE01812F0E946D
:101C30000D15DF91CF911F910895E1E0F0E0DF01F4
:101C400002C0AA0FBB1F6A95E2F7BD01DF0102C007
:101C5000AA0FBB1F4A95E2F7AD01462B01C0EE0F5C
:101C60002A95EAF7942F9823491302C08E2B0895E2
:101C7000E0958E230895242F462F682F8091080326
:101C80000E941D0E0E94FF0C08951F93CF93DF93B7
:101C9000C0910A0317E080910B03C817A1F0D0E0B0
:101CA0001C9FF0011D9FF00D1124E45FFC4F20816B
:101CB0003181428153816481758186810E94D00C7B
:101CC0002196C770E8CFDF91CF911F9108952091A1
:101CD000440330914503409146035091470360917E
:101CE00048037091490380914A030E94D00C0895E3
:101CF000CF93DF9380914A0382958F7009F04EC095
:101D000080914903882309F449C080910A034091D6
:101D10000B035091450360914403C0914603D09159
:101D2000470377E08417D1F190E0789FF001799F25
:101D3000F00D1124DF01A45FBC4F14962C91149771
:101D4000222349F111962C911197251324C02C912F
:101D5000261321C015962C91159721111CC012969F
:101D60002D913C9113972C1B3D0B283C310598F489
:101D700080914A038F70806180934A03EE5EFC4F2E
:101D800080818F708061808384E493E00E94600C86
:101D90000E94450E03C001968770C4CFDF91CF919A
:101DA000089520910A0390910B0357E02917A9F099
:101DB00030E0529FF001539FF00D1124E45FFC4F7F
:101DC0007181761306C07081781303C07581741316
:101DD00006C02F5F3F4F2770E9CF80E0089581E074
:101DE0000895A4E1B0E0E7EFFEE00C94712F8C01C0
:101DF00086E0F801DE011F9601900D928A95E1F7C9
:101E0000F8018481E58094E4A92E93E0B92E9091A5
:101E10004803911118C0882309F480C1EE20D9F13C
:101E2000C8010E94B90CF82E8823A9F187E0F801B7
:101E3000D50101900D928A95E1F7C5010E942E0906
:101E40000E94780E98C0F801C080D1808280938073
:101E5000F09049032091460330914703A401421BAF
:101E6000530BFF2009F406C1483C510508F0AFC0F0
:101E7000882309F455C180914A03282F207F90912F
:101E80004503222361F09D1509F462C0C8010E9438
:101E9000B90C811173C0C8010E94600C3FC19D1133
:101EA00015C0909144039C1111C0E1100FC08F70B8
:101EB000806180934A030E94670E84E493E00E944D
:101EC000600C80914A03F801868326C1E1103AC074
:101ED00040E06D2D8C2D0E94D10E40E06D2D8C2D9B
:101EE0000E94D10EE82E811117C1CF86D88A8F8526
:101EF00098890E94EF0D292F22952F70243020F40D
:101F00009F70223028F009C02A50223080F014C07F
:101F1000992349F0811107C013C0992321F0F801DA
:101F20009681907F69F0805E883030F409C0803FF0
:101F300038F0815F833020F0C8010E94600CEF2CE4
:101F4000FE2CEEC080914A03816080934A03E4C076
:101F5000909144039C119ACFE11098CFF8018683A9
:101F6000C8010E94600C87E0F801A4E4B3E001908E
:101F70000D928A95E1F70E94670ED2C0EE2009F417
:101F80008ACF20914A03822F82958F7090E002972A
:101F90008CF08091440390914503998788879B86B4
:101FA0008A86809148038C871D862E87CE010896ED
:101FB0000E94600C87E0F801A4E4B3E001900D9268
:101FC0008A95E1F70E94780E0E94670EA7C0909153
:101FD0004A03292F207FA1F4682D9A8A898AA601B5
:101FE0007A899E2D0E94C60C84E493E00E94600CC6
:101FF00087E0F50111928A95E9F70E94670E8CC07F
:10200000882309F48DC0809145038D1111C0809102
:1020100044038C110DC0E1100BC0F8019683C80178
:102020000E94600C87E0F50111928A95E9F778C06B
:10203000C8010E94B90C882309F42DCFEE2009F4C1
:102040002ACF20914A03822F82958F7090E00297C9
:102050000CF4B0CF80914403909145039A83898317
:102060009C828B82809148038D831E822F83CE01B8
:1020700001969ECF483C510508F040C0882309F4E2
:102080004DC0FE2CEE2009F406CF809145038D1142
:1020900027C0809144038C1123C090914A0390FD86
:1020A00016C0892F82958F70282F30E021153105B9
:1020B00071F0F80196832F30310509F451CF8F5F0D
:1020C000982F9295907F86818F70892B48CF87E0DB
:1020D000F801A4E4B3E001900D928A95E1F720C0E5
:1020E000C8010E94B90C811165CF80914A038160BB
:1020F00080934A03C8010E94600C12C0682D9A8A1E
:10210000898AA6017A899E2D0E94C60C87E0F50176
:1021100011928A95E9F72FCFF12C02C0FF24F39496
:102120008F2D6496ECE00C948D2FAEE0B0E0EBE9DF
:10213000F0E10C947A2F288739874A875B876C8770
:102140007D878E87CE0108960E94F10E882361F06C
:102150006C856623A9F1288539854A855B857D854F
:102160008E850E94D00C2CC087E0FE013896DE01DF
:10217000119601900D928A95E1F76C85662301F125
:1021800020910B0330E0C901019687709927409197
:102190000A0350E084179507E1F16D8397E0929F61
:1021A000D001939FB00D1124A45FBC4FFE01319666
:1021B00001900D929A95E1F780930B030E94450ED2
:1021C00017E080910A0390910B03891779F1189F0A
:1021D000C0011124845F9C4F0E94F10E882331F1CD
:1021E000E0910A031E9FF0011124E45FFC4F20815F
:1021F0003181428153816481758186810E94D00C36
:1022000080910A0390E001968770992780930A03D2
:10221000D8CF0E94990C10920B0310920A03E4E4A9
:10222000F3E087E0DF011D928A95E9F72E96E3E05F
:102230000C94962F809153038695869586950895E4
:10224000809153038770089590915303977081E0B4
:1022500009F480E0089580915F03089590915F03F1
:10226000892B80935F030895809590915F03892364
:1022700080935F03089510925F03089590915E0329
:10228000892B80935E030895809590915E03892346
:1022900080935E03089510925E03089508950E944E
:1022A0004E1108950E944F11089590915503292FC2
:1022B0002823821729F0982B909355030E945211DE
:1022C000089590915503292F282331F08095892373
:1022D000809355030E9452110895809155038823DD
:1022E00029F01092550380E00E94521108950F9337
:1022F0001F93CF93DF930091000110910101C091D2
:102300005F0380915E03C82B80915503882331F0D1
:10231000C82B0E944E2581110E946D11F801C083C7
:10232000C0910001D091010148E050E06BE473E0FE
:10233000CE010E94B62F892B59F088E0FE01ABE454
:10234000B3E001900D928A95E1F7CE010E94A92495
:10235000DF91CF911F910F9108950E9477110895F9
:102360000E944E1108950E94B01108959091540357
:10237000292F282331F080958923809354030E94CC
:10238000B31108950E944E1108959091A20392FFF7
:1023900011C098E0899F90011124262B20935303AC
:1023A0000E94110D809153038695869586950E9413
:1023B000C21108950E94110D08951092530380E0F8
:1023C0000E94C211089590915303809589238093B0
:1023D0005303282F277069F4981759F09091A2039E
:1023E00092FF07C08695869586950E941D0D0E94D6
:1023F000DD110895CF939091A20392FB222720F93B
:102400002817F9F0C82F892FC0FB82F98093A20307
:102410008091A1039091A2030E945D1282E00E942C
:10242000E3118091740380FF0CC01F92CF938BED5A
:1024300093E09F938F930E943A070F900F900F9015
:102440000F90CF9108958091A20382FB882780F995
:1024500091E089270E94FA11089581E00E94FA1103
:10246000089580E00E94FA1108956FEF7FEF80E0F9
:1024700090E00E940830089580E090E00E94D42F00
:10248000853E9E4F19F40E943F23089580E00895F1
:1024900082E090E00E94CC2F089583E090E00E94BB
:1024A000CC2F0895682F83E090E00E94EA2F0895D2
:1024B00084E090E00E94D42F0895BC0184E090E075
:1024C0000E9408300895AB01BC018FE090E00E94AB
:1024D000FC2F0895AB01BC0183E190E00E94FC2F2A
:1024E000089560E070E0CB010E946A12089560E0F8
:1024F00070E0CB010E9463120E9471120895A8E05F
:10250000B0E0E5E8F2E10C947B2F65EE7EEF80E031
:1025100090E00E94083060E082E090E00E94EA2FA4
:1025200081E0809309030E94521260E074E184E02C
:1025300090E00E94083060E086E090E00E94EA2F80
:1025400060E087E090E00E94EA2F40E050E0BA01AE
:1025500088E090E00E94FC2F60E083E290E00E941F
:10256000EA2F60E08CE090E00E94EA2F60E08DE0CE
:1025700090E00E94EA2F19821A821B821C821D821F
:102580001E821F82188648E050E067E170E0CE01AD
:1025900001960E94DA2F40E050E0BA018FE190E00E
:1025A0000E94FC2F80E00E9458230E948D230E94ED
:1025B00077122896E2E00C94972F0E947F120895DC
:1025C000682F8EE090E00E94EA2F0895A6E0B0E028
:1025D000ECEEF2E10C94792F0E94DB268C018091C5
:1025E0006003909161030817190781F019821A821C
:1025F0000E94DB26682F49815A81792F80E090E084
:102600000E94FB0810936103009360032696E4E0A8
:102610000C94952F0E94E7266093700370937103CA
:10262000809372039093730360936C0370936D03B4
:1026300080936E0390936F03089581E0089581E085
:1026400008950E941F13089508950E942413089569
:102650000E94241308950E94281308950E942413B1
:1026600008950E942E1308950E942413089580E473
:1026700099E20E94C5170E9434130E9431130895F5
:102680000E9425130E94241308950E943C12811178
:1026900002C00E94DD120E944812809374030E94BF
:1026A00058129093A2038093A1030E94E8170E94FE
:1026B0004D120E94E70C809108030E94FC0C0895C3
:1026C0000E94D2260E949D230E941B170E94451340
:1026D0000E94C3080E942B130895A6E0B0E0E3E730
:1026E000F3E10C946F2F0E941D13811103C00E940F
:1026F000E61262C00E94311722E6E22E23E0F22E9B
:102700005701D12CF501019111915F018D2D0E948E
:10271000101680279127D394F5E0DF1619F0892B46
:1027200089F302C0892B19F38091740381FD0E9403
:1027300019160E942113782E10E066246394812FCD
:102740000E9410164C01F701A080B180A826B9267E
:10275000A114B10449F100E0CC24C394D12CC501EB
:102760008C219D21892BC1F07720B1F009831A8338
:102770000E94DB269C838B836D8221E0C4018C2127
:102780009D21892B09F420E049815A816B817C814C
:102790008D81922F0E94FB080F5FCC0CDD1C0F3047
:1027A000F1F6F701918280821F5FF2E0EF0EF11CDB
:1027B000153029F60E940A130E943F200E94D0087B
:1027C0002696EEE00C948B2F1F93CF93DF930E94FD
:1027D0001215EC01C11580E5D807E8F5C11590E4A4
:1027E000D90708F0A8C0C03ED10530F5CD3CD105D1
:1027F00008F094C0C83AD10578F4C53AD10508F07C
:1028000083C0C130D10509F47CC008F4F2C0C430E3
:10281000D10508F0F1C0EDC0C33CD10508F0E9C016
:10282000C85AD0E0CC0FDD1FCC5ADE4F0990D881BA
:10283000C02DCE019464E1C0C11580E2D80708F034
:10284000CBC0C11591E0D90708F06BC0C83ED105D7
:1028500008F4D2C0CEC0C03682E5D80728F5C0340F
:1028600092E5D90708F079C0C03282E5D80708F0B0
:102870006CC0C11592E5D90708F481C04C2F46956C
:10288000469580E2489FA0011124C37021E030E00A
:10289000C90102C0880F991FCA95E2F7EA01C82B47
:1028A000D92BCE019D68A9C0C03A82E5D807B8F4FB
:1028B0008C2F8F71C03892E5D90708F07BC08695C0
:1028C000869590E2899F90011124C37081E090E089
:1028D00002C0880F991FCA95E2F79A6868C0C03C89
:1028E00082E5D80708F46DC0C03E92E5D90708F02C
:1028F00080C0CF71DD27DC2FCC27CE01806F906A9E
:102900007CC081E090E079C0C55AD0E0C657DE4F68
:102910008881C82FD0E0CE0190646FC0CE01906551
:102920006CC08D2F0E94AE15182FCE0199270E94E2
:1029300012151F715CC0CE0199270E941215CC2779
:10294000DF70D06A8C2B9D2B58C0CF71D0E0DC2F6C
:10295000CC27CE01816F906A50C08C2F8F718695E5
:10296000869590E2899F90011124C37081E090E0E8
:1029700002C0880F991FCA95E2F79C6818C08C2F77
:102980008F710E94AE1595E0D695C7959A95E1F79F
:10299000CF70D0E0DC2FCC27282F30E084FF05C09B
:1029A00084E0220F331F8A95E1F7D069CE01822B94
:1029B000932B23C090E0D82FCC27CE01846F906A50
:1029C0001CC08C2F8F710E94AE158F7190E0D82F94
:1029D000CC27CE01906211C08D2F8F710E94AE1551
:1029E000182FCE0199270E9412151F719062912B0A
:1029F00004C080E090E001C0CE01DF91CF911F9133
:102A00000895753038F46F3028F4462F672F0E94F0
:102A1000101C089580E090E008950E9401150E9426
:102A2000E41308958238910569F1B0F4813391057A
:102A300009F475C048F48932910509F467C08A32F7
:102A4000910509F471C008958533910509F459C0C1
:102A500089339105B9F00895833E910589F138F4E1
:102A6000803E9105D1F0823E910529F10895863E80
:102A70009105C9F1873E9105D9F1843E910509F090
:102A80006CC027C02091A10320FD57C021FD55C077
:102A90002091A20323FD5BC008958091A10380FDD6
:102AA00048C08091A20380FF48C08091A10384FDAB
:102AB00046C083EE51C08091A10382FF3CC0F5CF98
:102AC0008091A10382FD37C08091A20380FD35C0B3
:102AD000ECCF8091A20381FF36C08091A10384FDD9
:102AE0002EC087EE39C08091A10383FF2AC0F5CFA5
:102AF0008091A10383FD25C08091A20381FD23C0A5
:102B0000ECCF8091A10385FD22C01FC08091A1035D
:102B100085FD1BC08091A20383FF19C00AC080916C
:102B2000A10386FD16C017C08091A10386FD13C0C6
:102B300010C089E311C082EE0FC080EE0DC080E0AE
:102B40000BC086EE09C084EE07C085E305C089E2AC
:102B500003C08AE201C081E390E008959091A1034F
:102B600092FF10C041E0282F2471243009F040E08A
:102B700031E0282F2871283009F030E0431711F098
:102B80002CE0822793FF10C041E0282F24712431CC
:102B900009F040E031E0282F2871283109F030E0B9
:102BA000431711F02CE082273091A20330FF10C0B0
:102BB00051E0282F2171213009F050E041E0282F09
:102BC0002871283009F040E0541711F029E08227DD
:102BD00031FF10C041E0282F2171213109F040E080
:102BE00031E0282F2871283109F030E0431711F027
:102BF00029E0822794FD877E0895CF939C01205E73
:102C000032452032310540F4FB01C581C11105C0B8
:102C10008F710E94C90701C0C1E08C2FCF91089528
:102C2000E82FF0E0EE0FFF1FE355FC4F808191810C
:102C30000895A0E0B0E0EFE1F6E10C94712F80E0A0
:102C400094E09F938F930E943A078DEAE82E83E0E9
:102C5000F82E0F900F90812C912C9BEFA92E93E0D2
:102C6000B92E28EFC22E23E0D22E02EF13E0C0EFE0
:102C7000D3E09F928F92BF92AF920E943A07DF9269
:102C8000CF920E943A07F701819191917F010E94B2
:102C90009E089F938F931F930F930E943A07DF9391
:102CA000CF930E943A079FEF891A990AEDB7FEB7B2
:102CB0003C960FB6F894FEBF0FBEEDBFF5E08F1641
:102CC0009104B9F6CDB7DEB7ECE00C948D2F80EA15
:102CD0008A95F1F7089500C008950E946716089537
:102CE00008950E94701608950E94711608950E941A
:102CF000701608950E9477160895F894E82FE295CB
:102D0000EF70F0E031A1282F2F7081E090E001C03A
:102D1000880F2A95EAF7982F9095932391A392A173
:102D2000892B82A3789408950F931F93CF93DF93F9
:102D3000CCE9D1E089918F3F11F00E947D1681E0AE
:102D4000C13AD807B9F7CDE8D1E00CE911E0899193
:102D50008F3F11F00E947D160C171D07C1F7DF9100
:102D6000CF911F910F910895A0E0B0E0EAEBF6E15A
:102D70000C94742F8C01C62FD0E0CE0184569E4F48
:102D80006C01FC0190819F3F09F450C0B62EF8946D
:102D9000E92FE295EF70F0E081A19F7021E030E033
:102DA00001C0220F9A95EAF7822B81A382A1209578
:102DB000282322A378940E946B16EDE8F1E04CE9F9
:102DC00051E021E030E0E12CF12C61916F3F89F07E
:102DD000A62FA295AF70B0E090968C9190E06F70A6
:102DE00002C0959587956A95E2F780FD02C0C901FA
:102DF00002C080E090E0E82AF92A220F331F4E1724
:102E00005F0719F7F60180818F3F11F00E947D1650
:102E100061E0E114F10409F460E08B2D0E946D166D
:102E2000CC0FDD1FC00FD11FF982E882CDB7DEB70E
:102E3000E9E00C94902F0E9494168AE0EDEAF3E00A
:102E4000DF01982F1D929A95E9F7E3EAF3E0DF019D
:102E50001D928A95E9F785E00E946C170E947A1608
:102E60000895AAE0B0E0E7E3F7E10C94782F8E0133
:102E70000F5F1F4F8AE0F80111928A95E9F7F12C54
:102E80006F2DC8010E94B416F394F5E0FF12F8CF3D
:102E90004AE050E0B80183EA93E00E94B62F21E0B7
:102EA000009709F420E0892B41F08AE0F801A3EAB9
:102EB000B3E001900D928A95E1F745E06DEA73E089
:102EC00083EA93E00E946D17182F0E947416812FD9
:102ED0002A96E5E00C94942F0895EF92FF920F93B9
:102EE0001F93CF93DF937C018B01C42F222351F0DA
:102EF00081E0809377030E94DB2690937603809392
:102F0000750304C080917703811102C080E01CC06A
:102F100080917503909176030E94F3260597B0F394
:102F2000D0E0CC0FDD1FAE01B701C8010E94B62F63
:102F3000892B39F0AE01B701C8010E94C32F81E08F
:102F400001C080E010927703CDB7DEB7E6E00C94C5
:102F5000932F0E946D1308950E9472260E94A32948
:102F60000E9437130E94BD290E9460130E94CA2943
:102F70000E94CF290E94A9170E94F7290E94962734
:102F80000E94C6270E944013F3CF9093E3028093E0
:102F9000E20208950E943512089580E00E94101602
:102FA000817008950E9431172FEF86E791E021503C
:102FB00080409040E1F700C000000E9431170E945D
:102FC000CD17882321F00E94CA170E942827089550
:102FD0000E94D2170895809102011F928F938091D1
:102FE00003011F928F93809106011F928F9380910E
:102FF00007011F928F93809108011F928F938091F8
:1030000009011F928F9387E194E09F938F930E9411
:103010003A078DB79EB70E960FB6F8949EBF0FBEB7
:103020008DBF0895883220F58E3108F072C08B3044
:1030300091F1C0F4873009F0CCC081E080930901A0
:1030400084E1809308018AE0809307018EE18093F8
:10305000060188E08093030188E28093020189E7FA
:1030600095E0D4C0833109F44BC0843189F1B1C0FB
:103070008F3409F4ACC028F4893251F1883359F007
:10308000A8C0813531F008F4E6C0823509F4B5C036
:10309000A0C08FEFB3C08BE995E09F938F930E9400
:1030A0003A070E94EB171F9281E08F931F9288E0EE
:1030B0008F9384E994E09F938F930E943A078DB792
:1030C0009EB708960FB6F8949EBF0FBE8DBFA4C0E2
:1030D00088E995E09F938F930E943A070F900F9095
:1030E00080917C03882309F4B4C010927C03109271
:1030F0007B0310927A031092790310927803BBC07D
:103100008AE895E09F938F930E943A070E94EB17FD
:1031100081C08D5180937C03833031F170F4813014
:10312000D1F0823009F03FC088E091E090937B03BA
:1031300080937A038EEA91E01FC0853059F108F13F
:10314000863089F582E091E090937B0380937A0347
:1031500089EE91E011C089E091E090937B03809328
:103160007A0385EA91E008C087E091E090937B03C1
:1031700080937A038AEB91E09093790380937803AC
:103180001CC086E091E090937B0380937A0387ECE8
:1031900091E0F2CF83E091E090937B0380937A03F8
:1031A00086ED91E0E9CF10927C0387E895E09F934C
:1031B0008F930E943A070F900F9080917C03882391
:1031C00009F459C01F928F9383E895E00DC08AE0FF
:1031D00015C086E795E01AC097FF4BC0108280812A
:1031E0001F928F9380E795E09F938F930E943A07F9
:1031F0000F900F900F900F900FC081E0E0917A0335
:10320000F0917B03309749F58DE695E09F938F937E
:103210000E943A070F900F9020917C03222359F1CE
:103220008091780390917903009711F481EA91E0FD
:103230009F938F931F922F9384E695E09F938F9394
:103240000E943A070F900F900F900F900F900F90E1
:103250001AC080E0089586EFD1CF2081082E000C9F
:10326000990B820F911D8F3F910509F00CF4B4CF9B
:103270008FEF8083B4CF80E695E09F938F930E9479
:103280003A070F900F9081E00895CF93C82F1F92B7
:103290008F9381EB95E09F938F930E943A0781E093
:1032A00001C0880FCA95EAF70E94E70C0E94990CAA
:1032B0000F900F900F900F90CF910895EF92FF9283
:1032C0000F931F93CF93DF938B3109F408C108F05C
:1032D0009BC08B3009F4C2C008F07DC0863009F471
:1032E000C0C020F4853009F4D2C073C1873009F41E
:1032F000D7C0883009F06DC10E944D121F928F9384
:1033000089E399E09F938F930E943A070E944812A5
:1033100083FB992790F91F929F9382FB992790F93D
:103320001F929F9381FB992790F91F929F93982F4B
:1033300091701F929F931F928F9380EF98E09F93BD
:103340008F930E943A070E94581293FB222720F97C
:103350001F922F9387FB222720F91F922F9386FB22
:10336000222720F91F922F9385FB222720F91F92F5
:103370002F9384FB222720F91F922F9383FB222770
:1033800020F91F922F9382FB222720F91F922F935F
:1033900091FB222720F91F922F93292F21701F9232
:1033A0002F9381FB222720F91F922F93282F217022
:1033B0001F922F939F938F9381EF97E09F938F930B
:1033C0000E943A078DB79EB78A960FB6F8949EBFB3
:1033D0000FBE8DBF41C0803109F4ABC020F48E30E8
:1033E00009F490C0F6C0863109F4C6C0893109F0ED
:1033F000F0C08EEF91E09F938F9381E296E09F93D0
:103400008F930E943A07B3C08A32E1F060F48732AA
:1034100009F4DBC028F48E3108F4DBC08D51D6C02E
:103420008932A9F1D6C0833448F48A3308F0CBC07E
:10343000853309F4CAC0883389F0CBC0833409F4DA
:10344000C4C0C7C084EE99E09F938F930E943A074F
:103450000E94DD120F900F90C1E0C4C08BE496E093
:1034600063C080917403817F8E7F8093740384E2B4
:1034700096E09F938F930E943A0780EE99E09F9386
:103480008F930E943A0781E080937D0370C084ECA3
:1034900099E09F938F930E943A070E94EF07DACF3B
:1034A00080917403C82FC095C170C0FB80F98093D0
:1034B0007403CC2339F088EB99E09F938F930E949B
:1034C0003A074FC08BEA99E09F938F930E943A0787
:1034D00080917403897F877F80937403BBCF809131
:1034E000740381FBCC27C0F991E0C927C0FB81F9A7
:1034F00080937403CC2319F08EE999E029C080E908
:1035000099E012C08091740382FBCC27C0F991E04E
:10351000C927C0FB82F980937403CC2319F081E89A
:1035200099E016C081E799E09F938F930E943A0734
:1035300091CF8091740383FBCC27C0F991E0C92718
:10354000C0FB83F980937403CC2371F085E699E086
:103550009F938F930E943A078091740381608093B8
:1035600074030F900F903EC088E599E0DDCF0F9077
:103570000F900F900F9070CF0E94E726162F072F05
:10358000F82EE92E0E944A26D82F0E942A26C82FFC
:103590000E949924EF92FF920F931F931F92DF9343
:1035A0001F92CF931F928F9386EB95E09F938F93FB
:1035B0000E943A078DB79EB70C960FB6F8949EBF3F
:1035C0000FBE8DBF49CF895301C080E00E944519CD
:1035D00043CF86E599E09F938F930E943A070F901F
:1035E0000F90C0E08C2FCDB7DEB7E6E00C94932FA0
:1035F00080E008950E94F81A0895CF93C82F809113
:103600007D03813079F040F0823009F052C08C2F78
:103610000E94121881E053C00E942B11823209F0DF
:103620004AC004C00E942B11823261F48C2F0E9488
:10363000FA1A811104C08C2F0E945E1938C081E0F3
:1036400090E035C08C2F0E94F81A81112FC0C43130
:1036500009F158F4CB3069F0C031F9F482E080937D
:103660007D0388E30E94121821C0C93299F0C83343
:10367000A1F484E296E09F938F930E943A078DEA2B
:1036800095E09F938F930E943A070F900F900F90B1
:103690000F900CC010927D0310C08BEA95E09F93B1
:1036A0008F930E943A070F900F9007C081E08170BE
:1036B00006C010927D0380E002C080E0F8CFCF9179
:1036C000089584E0089550E0440F551F2EE1629F55
:1036D000400D511D11249A0166E9869F200D311D70
:1036E0001124C901889608950F931F93CF93DF93F8
:1036F0008430A0F4653090F44F3080F40E94631B56
:103700008C010E94CC2F90E0D82FCC27C8010196C5
:103710000E94CC2F9E01282BC90102C080E090E0BE
:10372000DF91CF911F910F9108950F931F93CF9326
:10373000DF93843080F4653070F44F3060F4E90139
:103740000E94631B8C016D2F0E94EA2F6C2FC80111
:1037500001960E94EA2FDF91CF911F910F9108955A
:103760001F93CF93DF93D0E0C0E010E0412F6C2F88
:103770008D2F0E9443079C01412F6C2F8D2F0E949B
:10378000951B1F5F1F3091F7CF5FC53071F7DF5F6B
:10379000D43051F7DF91CF911F910895EF92FF92AE
:1037A0000F931F93CF93DF93EA017A01E60EF71E82
:1037B0008C01C8018896CE15DF0569F0083522E036
:1037C000120720F40E94CC2F888301C01882219612
:1037D0000F5F1F4FEECFCDB7DEB7E6E00C94932F0F
:1037E000EF92FF920F931F93CF93DF93EA017A0139
:1037F000E60EF71E8C01C8018896CE15DF0559F03C
:10380000083522E0120718F468810E94EA2F2196F9
:103810000F5F1F4FF0CFCDB7DEB7E6E00C94932FCC
:10382000843038F4653028F44F3018F40E94741B4B
:10383000089580E090E0089580E1089580E891E0A7
:103840000895EF92FF920F931F93CF93DF93EA01B6
:103850007A01E60EF71E8C01C80180589D4FCE15E7
:10386000DF0569F0003821E0120720F40E94CC2F18
:10387000888301C0188221960F5F1F4FEDCFCDB70F
:10388000DEB7E6E00C94932FEF92FF920F931F9315
:10389000CF93DF93EA017A01E60EF71E8C01C8018F
:1038A00080589D4FCE15DF0559F0003821E01207F2
:1038B00018F468810E94EA2F21960F5F1F4FEFCF07
:1038C000CDB7DEB7E6E00C94932FCF93DF93C0E83B
:1038D000D2E060E0CE010E94EA2F2196C11584E07B
:1038E000D807B9F7DF91CF910895A8E0B0E0EBE7F2
:1038F000FCE10C94712FF82E8FE08F1508F474C042
:103900008FEF93E00E94CC2F81116EC000E812E08F
:10391000FF2071F0011594E0190709F465C0C80192
:103920000E94CC2F811101C0FA940F5F1F4FF0CF7E
:10393000FE0131966F0188E011928A95E9F77801CE
:10394000FFEFEF1AFF0AC8010E94CC2F89831A8269
:10395000882309F449C0813009F040C0580182E051
:10396000A80EB11CC7010E94CC2F8A838823E1F1E5
:103970009FEF980F933060F4780193E0E90EF11C0B
:10398000C5010E94CC2F8B83882371F11C8226C035
:10399000843019F54E01E3E08E0E911C02E010E038
:1039A0007501FFEFEF1AFF0AC5010E94CC2FF40149
:1039B00081934F018823C1F08C3741F4E2E0F0E0BD
:1039C000EC0FFD1FE00FF11F108208C00F5F1F4FAB
:1039D00057010730110521F707C0750160E0C601E6
:1039E0000E94DF218701ABCF2896ECE00C948D2F4D
:1039F000CF93DF9386319C4709F5EB010E942B1191
:103A00009D81992371F08A7A91E009F490E0909376
:103A10007E03811102C089E201C085E30E949825DE
:103A200009C080917E03811102C089E201C085E353
:103A30000E94A0250E94AD1180E001C081E0DF91CD
:103A4000CF910895CF93DF93FC01DB0115968C9104
:103A5000882309F4DDC09F0130572332310508F077
:103A6000D8C0EF010E9458129093A2038093A10343
:103A7000FE01E150F047E232F10520F4EE59FF4F2C
:103A80000C945E2F8091A1038160AAC08091A20353
:103A90008860B2C08091A1038260A2C08091A1031E
:103AA00020C08091A10388609BC08091A2031EC0AA
:103AB0008091A2038260A0C08091A103806190C028
:103AC0008091A10380628CC08091A103806488C032
:103AD0000E94990C8091A103806882C08091A1030B
:103AE000886084607DC08091A2038260816084C010
:103AF0008091A1038E7F74C08091A203877F7CC0D8
:103B00008091A1038D7F6CC08091A10320C0809122
:103B1000A103877F65C08091A2031EC08091A2038C
:103B20008D7F6AC08091A1038F7E5AC08091A103CE
:103B30008F7D56C08091A1038F7B52C00E94990C4B
:103B40008091A1038F774CC08091A103877F8B7FE9
:103B500047C08091A2038D7F8E7F4EC08091A103CC
:103B600082FB222720F991E0922790FB82F990FBBB
:103B700083F936C08091A203982F909591708E7F23
:103B8000892B90FB81F938C08091A10386FB222705
:103B900020F991E0922790FB86F922C00E94990CAF
:103BA0008091A10387FB222720F991E0922790FBC7
:103BB00087F916C081E001C080E00E94E0121EC0BB
:103BC0008091A10384FB222720F991E0922790FBAA
:103BD00084F906C08091A103982F909590FB80F9FD
:103BE0008093A1030BC08091A20383FB222720F9BD
:103BF00091E0922790FB83F98093A2038091A10327
:103C00009091A2030E945D120E94990C80E001C075
:103C100081E0DF91CF910895282F35EB2303C00178
:103C2000112497FF03C08058910902C080589F4F0C
:103C3000892F08958091850380FF06C06091070158
:103C400070E0660F771F26C081FF04C060910701F6
:103C500084E005C082FF07C06091070188E0689F8B
:103C6000B001112417C0909184039923D1F0609181
:103C70000601961788F72091070188E0289F900198
:103C80001124929FA001939F500D112470E0CA014E
:103C90000E944A2F6038710540F46115710519F4CE
:103CA00006C068E070E0862F08958FE7089581E0F0
:103CB00008958091850380FF08C06091030170E042
:103CC000759567957595679521C081FF06C06091D0
:103CD000030170E07595679519C082FF04C060917B
:103CE000030170E010C090918303992399F06091D3
:103CF00002019617A0F780910301899FC00111244A
:103D000070E00E944A2F6038710540F4611571051A
:103D100019F406C061E070E0862F08958FE70895DA
:103D200081E008958D3C21F40E941A1E819504C003
:103D30008E3C29F40E941A1E8093890308958F3CBB
:103D400021F40E941A1E819504C0803D29F40E942E
:103D50001A1E809388030895893D19F40E94591E04
:103D600005C08A3D31F40E94591E819580938A03D3
:103D700008958B3D21F40E94591E819504C08C3D0D
:103D800029F40E94591E80938B0308959FE2980F97
:103D9000983078F421E030E0A90102C0440F551FAB
:103DA0009A95E2F7CA0190918703892B8093870344
:103DB00008958D3D21F48091850381600BC08E3D77
:103DC00021F480918503826005C08F3D29F48091A4
:103DD000850384608093850308958D3C39F4909128
:103DE000890397FF35C01092890359C08E3C29F48E
:103DF000909189031916BCF32BC0909188038F3CD6
:103E000029F497FF25C01092880349C0803D19F41A
:103E10001916CCF31DC090918A03893D29F4191617
:103E2000BCF410928A033BC08A3D19F497FF10C07E
:103E3000F8CF8B3D39F490918B0397FF09C0109216
:103E40008B032DC08C3D21F490918B031916BCF38C
:103E50009FE2980F983080F421E030E0A90102C081
:103E6000440F551F9A95E2F7CA01809590918703F8
:103E700089238093870313C08D3D21F480918503AE
